:020000040000FA
:06000000000080EF00F09B
:0400080010EF00F005
:0400180010EF00F0F5
:10002000AE50076E06660CD04E0E076204D0096A09
:10003000062A086A1100520E07621100092AF8D731
:100040000D0E07624AD0086601D04DD0040E08603C
:100050004AD0E55008060844F92614D00CD0E550E3
:100060000A6E0A0EE502F3500A26010EE75C3BE138
:10007000640E0A2609D0E5500A6E0A0EE502F35016
:100080000A2602D0E5500A6E0A52D8B42CD00A06CD
:100090000ABE29D0026A0A3202320A3202320A3217
:1000A00002320242023A022A0F0E0A16010E0C6EAA
:1000B000020602E00C46FCD7096608D00C1E0A5066
:1000C000EB500C160A500CC0EBFF0DD00A50EB5051
:1000D0000C120A500CC0EBFF06D0075009D803E3FE
:1000E000E66E082A1100066A086A10EE1EF011007A
:1000F000C60F03E20A0F01E31200D89012001000AD
:10010000730ED36E896AFF0E926E8A6AFF0E936E2B
:100110008B6A900E946E8C6AFF0E956E8D6A000E3F
:10012000966EC26A0F0EC16ED08E070EB46EA66AAE
:10013000040EAC6E330EAF6EAB8E9D8A9F8AAB8879
:10014000066A006A036A046A100E026E00EE0EF080
:10015000EE6A022EFDD700EE0EF010EE1EF09E6A43
:10016000C00EF26E82A83BD000663DD0801C19E024
:10017000036201D0F7D739D8801C036E016A056A83
:10018000052A05620BD00150A96EA69EA680A85034
:10019000EB1C0D6E0D460D44836EE4D7012A054617
:1001A000F0D7036A811C046201D0DCD71ED8811C01
:1001B000046E016A056A052A05620CD00150080F19
:1001C000A96E0000A680A850EB1C0D6E0D460D44D4
:1001D000836EC8D7012A01B6C5D70546EDD70052B0
:1001E000C5E108D8C3D70AD8C1D7140E0B6E0B2EA1
:1001F000FED712008280956A002A120095688290CC
:04020000006A12007E
:020000040030CA
:0E000000FF080200FF8181FF0FC00FE00F40DC
:0200000400F00A
:100000000A0B08090E0F0D0C000201030405060778
:00000001FF
